:1000000000308A001B2900008512051000344C3096
:100010008400000803191B280130A100A001A00BD7
:100020000F28A10B0E284A30A000A00B15280000B5
:100030000000800B0C280034480883169B001C1419
:100040001A088312A1000034260883169B0083122D
:100050004C0883169A001C1555309D00AA309D004F
:100060009C14831283169C1C372883123228831217
:1000700083161C118312A60A003485160230CC00A8
:1000800007200034851205140330CC0007201F140C
:1000900000341F08F339CE004D0DA000A00DFC3038
:1000A000A00520084E049F001030A000A00B562889
:1000B00000009F149F185A280C13CF011E08CE0071
:1000C000D100D001A30183161E0883125007A1009E
:1000D0000318A30A5108A3072308A20000349F13A2
:1000E0000330CD0049201E08A10000346F202108F4
:1000F000453C031C7F280130A10081288128003065
:10010000A10000343F08CD003E08BF004D08BE00EE
:100110004C08BF063F0EA0000F30A0052008BF0608
:100120003F0EA000F030A0052008BE063F0CA00046
:10013000A00CA00C1F30A0052008BE063F0EA0009A
:10014000F030A00520080310A00D2008BF060034E1
:1001500005101F1000349F170034B20A3208283CE3
:10016000031DB4281030B20000340F1CB528323003
:100170008E028F010034B520C91FC0280514C12884
:100180000510B520491FC6280514C7280510B5203D
:10019000C91ECC280514CD280510B520491ED2282B
:1001A0000514D3280510B520C91DD8280514D92851
:1001B0000510B520491DDE280514DF280510B520DF
:1001C000C91CE4280514E5280510B520491CEA28B7
:1001D0000514EB2805102808023C031DF3288E03A4
:1001E0008E03A801F428A80A00344908C802480868
:1001F0000F3C0318FD280F30C8002B08A00003197E
:1002000006290310CB0CCA0CA00B01294A0EC90009
:100210000F30C905490ECC00F030CC0548080F3925
:100220004C04A1000034A50A2508283C031D1A2906
:100230001030A500003484011F3083050730831679
:100240009F00073083129F001030A500A7018B1379
:100250008B1B272904201E3083168500073083124C
:1002600099001E3083169F00843083129F000B304C
:10027000A00007308101813084000008F039073880
:10028000800064000008F039200480006400013020
:10029000CC000720831683168312FF238316900059
:1002A000831283120C30C8001C2021086C3C0319F7
:1002B00078290230A600CC012420CC012420CC01D6
:1002C0002420CC012420B930CC0024205E30CC0086
:1002D00024202030CC0024201330CC0024200230F5
:1002E000CC0024208430CC0024206C30CC0024208E
:1002F0003D202830CC00072004206400C101C20149
:1003000042200330C200E830C100CB01CA014108DD
:1003100042040319A629640041080319C203C1035A
:100320000530CC0007204B084A06013C031DA029DC
:100330004630CC00072064005030CC000720A729AD
:100340004B08CA0076202108CB008729112A6400B7
:100350004B08CA0076202108CB004A06013C031D49
:10036000B5296430CC000720A7294B084A04003A7D
:10037000031DC4297620A108031DC0296400BA29E1
:100380003230CC000720C5298529BE01BF010630C7
:10039000B300B31BE929B1010830B200B208031958
:1003A000DE2964006430CC0007200310B10C7620F5
:1003B000A108031DDC29B117B203CE293308063C7E
:1003C000433E8400310880003108CC008220B30312
:1003D000C9296400BE08031D112ABF08031D112A84
:1003E0004308A600023C0319052A2608083C031D01
:1003F000042AC5080319002A2030CC002420032A2F
:100400000830CC002420052A112A4408CC002420DE
:100410004508CC0024204608CC0024204708CC0006
:1004200024200A30C8001C202108B000B00803199D
:100430001C2A2330A9001E2A0B30A900A820C101C4
:10044000C301C401C501C601C70164000B30C80067
:100450001C202108F039B100B10E0130C500C601E1
:100460003108A0000319392A0310C50DC60DA00BD1
:10047000342A3108033C03183F2A0730C7000B30E9
:10048000C8001C2021080739AB000130C2002B082E
:10049000A10003194F2A0310C20DA10B4B2A6400BF
:1004A000812AC101420841020318A62BAD01640054
:1004B0003F084705C300C40144084602031C812AC3
:1004C000031D662A450843020318812A2D0F692A55
:1004D000782A8316961583120B1064002B30A00027
:1004E000A00B702A0B1C752AAD0A83169611831275
:1004F00064006300000000000000C30A0319C40A7E
:100500005C2A4220AB200130CD0049202208C900DE
:100510002108C8003130CB006630CA00CC014B1B2B
:10052000992A4808CA024908031C490FCB02CC0A81
:100530008F2ACC034C08A1002108AC003C082D02F6
:100540000318A42A2D08BC002D083D020318AA2A6E
:100550002D08BD00A3012D08BA070318BB0A230804
:10056000BB07AB200230CD0049202208CA00210879
:10057000C9000130CD0049202208CC002108CB0061
:10058000C90DCA0DC90DCA0DC90DCA0DC90DCA0DB7
:10059000C90DCA0DC90DCA0DC90DCA0D8030C905D6
:1005A000C8014C084A02031CE32A031DDB2A490840
:1005B0004B020318E32A4B08C9024C08031C4C0FDA
:1005C000CA02C80AD12A3430C8024808A10021084A
:1005D000AE00300BF52AA3012E08A000A01BA30338
:1005E000B8070318B90A2308B90764006F20210867
:1005F000AF003008023C031D102B36082F020318F1
:10060000032B2F08B6002F0837020318092B2F08D9
:10061000B700A3012F08B4070318B50A2308B507CC
:10062000A820640064003D2090018E018F010130FC
:100630009000A80127088038AA00BE01BF01290840
:10064000CC0082202A08CC0082200230B20032087E
:100650000B3C031C342B3208C8001C202108C800A6
:10066000CC008220B20A272B2C08CC0082202D0837
:10067000CC0082202E08CC0082202F08CC008220C3
:10068000CC018220B0080319532B2508B200320890
:10069000C8001C202108C800CC008220AD202508FD
:1006A0003202031D472B6400B2013208093C031CCF
:1006B0005E2BAA30C900BB20B20A552BA530C90059
:1006C000BB202908C900BB202A08C900BB20023072
:1006D000B20032080B3C031C762B3208C8001C20E9
:1006E0002108C800C900BB20B20A692B2C08C90028
:1006F000BB202D08C900BB202E08C900BB202F0835
:10070000C900BB20C901BB20B0080319952B2508DF
:10071000B2003208C8001C202108C800C900BB2054
:10072000AD2025083202031D892B3E08C900BB20DD
:100730003F08C900BB20C901BB200420A70A270825
:100740003F3C0318A42BA701C10A522AB008031981
:10075000F82B2508A6003D08C8003C08C9003B0846
:10076000CB003A08CA00F5202108C800CC0024209C
:10077000132164002508A600300BDE2BB91BC12B0A
:10078000C62BB809B909B80A0319B90A2B08A00081
:100790000319CF2B0310B90CB80CA00BCA2BB91B33
:1007A000D22BD72BB809B909B80A0319B90A3808E6
:1007B000A1002108C800CC002420EB2B3708C8007A
:1007C0003608C9003508CB003408CA00F5202108D6
:1007D000C800CC0024201321FF30BC00BD01BB01A8
:1007E000BA01B901B801FF30B600B701B501B401D3
:0407F000512A630027
:02400E008C3FE5
:00000001FF
